:03000000021149A1
:03000B000200A54B
:03002B000202AE20
:03005B0002040C90
:030073000203E69F
:1000800002030406080C10182030406080040608A3
:100090000C10182030406080A0C00D0D0405060D26
:1000A0000503030302C2AFC0D0C0E020620C206889
:1000B00002419D306602415DE47385258AC262E596
:1000C00025F4700221242068022111207210758B02
:1000D00000D0E0D0D0C292C291C290D2AF32C292D0
:1000E000C291C2907406D5E0FDE53C1420E21520D3
:1000F000E10D207D02D295307D02D293020121D202
:1001000094020121207D02D293307D02D29502011A
:1001100021758B00D0E0D0D0C292C291C290D2AFF4
:1001200032758B00D0E0D0D0D2AF32419DE5256052
:100130000A207D02D292307D02D290C291419DE58B
:10014000256002D291207D02C290307D02C2924190
:100150009DE525600A207D02D290307D02D292205A
:100160007D02C292307D02C290419D207D02C293E9
:10017000307D02C295207D02C295307D02C293740B
:1001800006D5E0FDE525600A207D02D292307D0291
:10019000D290C291419D207D02C293307D02C295D2
:1001A000C2947406D5E0FDE525600A207D02D29256
:1001B000307D02D290C291419DC294207D02C293B3
:1001C000307D02C2957406D5E0FDE5256002D2912E
:1001D000207D02C290307D02C292419DC294207D5A
:1001E00002C295307D02C2937406D5E0FDE525601C
:1001F00002D291207D02C290307D02C292419D20A8
:100200007D02C295307D02C293C2947406D5E0FD92
:10021000E525600A207D02D290307D02D292207DB9
:1002200002C292307D02C290419D207D02C2953073
:100230007D02C293207D02C293307D02C295740676
:10024000D5E0FDE525600A207D02D290307D02D206
:1002500092207D02C292307D02C290419D30723D5B
:10026000E53C20E21A20E129207D02C293307D0284
:10027000C295207D02C295307D02C29302029D206C
:10028000E1E6207D02C293307D02C295C294020253
:100290009DC294207D02C295307D02C293E525F473
:1002A000F58A758B00D262D0E0D0D0D2AF32C2AF27
:1002B000C2AD53E6EFC0D0C0E0D2D3D2AFC2CEE5DC
:1002C0002960072074461529610C78007900E580C3
:1002D000307E01F430E40278FF53DACF207E03430E
:1002E000DA20307E0343DA10C2D8C271E580307E56
:1002F00001F430E40279FFC3E89970CE30610375F0
:1003000029182074037529188859D270E52A6004C9
:10031000152A611C20740543DA01C2D820700261DD
:1003200083A859206102C2702074367982B70431E3
:10033000C3E894F0400374F0F8E8C4540F28F87947
:1003400084B703026161C313C3138721200802C36A
:1003500013200A06C3C898F8616128F8500374FF97
:10036000F88822306915E5222408F5225003752209
:10037000FFC3E522955E4003855E227882B60418AD
:10038000852224A824C3E524955E4002A85EC3E824
:1003900095604002A8608825C3E52594404002D2BC
:1003A0006420CF0CD0E0D0D0C2D343E610D2AD321F
:1003B000C2CF7801E52960053074021529C3E559DB
:1003C00094014005755C0061DA755D00756400E5B7
:1003D0005C2401F55C5003755CFFD0E0D0D0C2D343
:1003E00043E610D2AD32C0D0C0E0C2AF53917F53CC
:1003F000E67FC260759100C3E49550F594E4955191
:10040000F595759104D0E0D0D0D2AF32C2AF53E6AB
:10041000EFC2ADC0D0C0E0C0F0D2D3D2AFA8FBA92C
:10042000FCC2D8307102817353DACF207E0343DAE5
:1004300010307E0343DA20D271E580307E01F42053
:10044000E402814A88268927C1AF53DACF207E0390
:1004500043DA20307E0343DA10C2D8C2713074020E
:10046000C19B7800E580307E01F430E402C19B88B6
:0F04700059C18253DACF207E0343DA20307E0356
:10047F0043DA10C271206102A14353DACF207E0309
:10048F0043DA10307E0343DA20C2D8D27188548900
:10049F0055C3E89552F8E99553F9E4FB7E027A00CB
:1004AF00C3E8948CE994005005755800A133C3E854
:1004BF0094C8E994005008E4D2E4FB7A0AA110C36F
:1004CF00E89468E994015008E4D2E3FB7A0FA11095
:1004DF00C3E894D0E994025008E4D2E2FB7A1EA15B
:1004EF0010C3E894A0E994055008E4D2E1FB7A3CEC
:1004FF00A110C3E89498E994085008E4D2E0FB7A7D
:10050F00787E00C3E89556FCE99557FD30E708EC77
:10051F00F42401FCEDF4FD755800C3EC9AED9E50E8
:10052F000375580188568957A854A955885289537D
:10053F007802C182C3E89526F8E99527F9307C0245
:10054F00C166307B02C166307A02C15F207502A19D
:10055F0066E9FDE8FCA185E9C313F9E813F83079E2
:10056F0002C15FE9C313F9E813F8307802C15FE9FC
:10057F00C313FDE813FC206126C3EC941CED940219
:10058F004002A19CED7018C3EC94C850120528C30B
:10059F00E528940A5002C19B755900D270C19BE5A2
:1005AF0028600215287400207F0B7888E67896B4AF
:1005BF000302789EE624FAFEE43400FFC3EC9EFCAF
:1005CF00ED9FFD92087888E6B40327A20850092012
:1005DF007D20C2AFD27DA1EE307D17C2AFC27DC2EA
:1005EF0092C291C290C293C294C295206902D26BFB
:1005FF00D2AFA2085017E6B4030DECF42401FCEDC2
:10060F00F43400FD02061C78007900C1667888E694
:10061F00B40315EC33FCED33FDC3EC940AFCED94FD
:10062F0000FD50047C007D00C3EC94FFED9400406E
:10063F000678FF7900C166EC856FF0A4C5F0A2F7CC
:10064F0033F87900400302068278FF7900020682B0
:10065F00E9C313F9E813F8307C0EE9600278FFC3A1
:10066F00E81338F8E43400F9C3E894FFE994004044
:10067F000278FF8859D270206102C19B741FF45514
:10068F002F4BF52FC274E42B7002D27475291830DA
:10069F00740375290A306102C1AF20740353DAFE67
:1006AF00752A06307403752A0AD0F0D0E0D0D0C274
:1006BF00D3D2AD43E6103279010206E47903020684
:1006CF00E4790A0206E4791E0206E479640206E47C
:1006DF0079C80206E47817E4D5E0FDD8FAD9F622F6
:1006EF007A147B7802070B7A107B8C02070B7A0D3A
:1006FF007BB402070B7A0B7BC802070BAC25752561
:10070F00017902B27DE4C294D5E0FDE5256002D205
:10071F0091D5E0FDC291D5E0FDD294D5E0FDE52560
:10072F00600A207D02D292307D02D290E570D5E032
:10073F00FD207D02C292307D02C2907496D5E0FDFD
:10074F00D9C1EAF8D5E0FDD8FBDBB1C2948C2522E4
:10075F00C37C007D0075F00005F0EA33FAEB33FB44
:10076F0050F6EB13FBEA13FAC3E9FFE8FEE89AF839
:10077F00E99BF95004EFF9EEF8B3EC33FCED33FDE0
:10078F00D5F0DFEDF9ECF822E889F08A20D2D4F821
:10079F00A9F07B0030F70B7BFFF42401F8E9F43468
:1007AF0000F9E88520F0A4ADF0F8E98520F0A4AFBA
:1007BF00F0FEED2EF974003FFA7C04C3EA13FAE958
:1007CF0013F9E813F8DCF48BF030F70AE8F424019E
:1007DF00F8E9F43400F9E889F0C2D4F8A9F02278E6
:1007EF0082B6040302084BC3E55994014003020883
:1007FF0013852224E4F53EF53FF540F541F542F52A
:10080F004702084B7882E6FC754701E522F523780D
:10081F003879C7AA3AAB3BC3EB13FBEA13FAEC14D4
:10082F006013C3EB13FBEA13FAEC14146007C3EB6A
:10083F0013FBEA13FA12075F883E893F22E54760F0
:10084F0034C3E53E9523F8E53F9400F9500CC3E817
:10085F009480E994FF4016020880C3E8947FE994DE
:0F086F00005003020880787F79000208807880AB
:10087E0079FF8843894422E5476058E5432540F8CF
:10088E00E5443541F9854420E4300701F43542FA58
:10089E0030E709C3EA94F040150208C2C3EA940F88
:1008AE0050030208C278FF79FF7A0F0208C278005F
:1008BE0079007AF0C3E524955E5006E524600901BF
:1008CE00DBE54420E70D01DBE54430E7068840898F
:1008DE00418A4222E547700302094678A1E6FAC32F
:1008EE00E54333F8E54433F9120797E930E70BC3D4
:1008FE00E89480E994FF4013211DC3E8947FE994A6
:10090E00005002211D787F7900211D788079FFE843
:10091E0020E715C3E52398F84009C3E89401400386
:10092E000209447801020944E8F424012523F84021
:10093E000302094478FF884522E54770030209A99E
:10094E0078A2E6FAA841A942120797E930E70CC34C
:10095E00E89401E994FF4016020980C3E894FFE988
:10096E009400500302098078FF7900020980780113
:10097E0079FFE920E715C3E54598F84009C3E894E7
:10098E000140030209A778000209A7E8F424012513
:10099E0045F840030209A778FF88242278FFC26435
:1009AE00E52D5406702FD264C3E53B940A4009C36B
:1009BE00E52594405002C264E53B601974FF853B07
:1009CE00F0848537F0A4F8C5F0600278FFC3E8958F
:1009DE00615002A8618860227883E6F520120F54D8
:1009EE0075E8901206C675E890E5E820ECFBA8BD08
:1009FE00A9BE121002756BAF756C00C3740013FDA7
:100A0E0074AF13FC74AF2CFC74003DFDECFAEDFBDF
:100A1E00C3E89AE99B4014E56B24AFF56BE56C34A3
:100A2E0000F56CEA2CFAEB3DFB80E5AE6BAF6CC3C8
:100A3E00E56C13F9E56B13F8C3E913F9E813F8E560
:100A4E006B28F569E56C39F56A7A03C3E913F9E8A1
:100A5E0013F8DAF7AA201A7009756B00756C00028C
:100A6E000A801AEA6008EE28FEEF39FFDAF88E6B7C
:100A7E008F6C2275E890227883E6FFE5E820ECF78C
:100A8E00A8BDA9BE056DC3E56D94084052756D00F5
:100A9E00E9FA79A0E76044EA7007E56E601B020A86
:100AAE00BBC3E8956E6010E56E5006600C14020A2A
:100ABE00C70460F9020AC7E56EF56EC39458401B71
:100ACE00755EC0C394044013755E80C39404400BDE
:100ADE00755E40C394044003755E0075BB0322EF40
:100AEE00C39401601BC3E894FFE994035012C3E85A
:100AFE00956BE9956C5009E55E601A155E020B2345
:100B0E00E55EF46010055E7888E6B40308E55E24C1
:100B1E00044002F55EA85EC3E524985002A824C3E3
:100B2E00E8955F400AA85FE55FF46003855F5E7934
:100B3E0082B70402614EC3E895604002A860882522
:100B4E00E56DB4070375BB1022743279A387F0A448
:100B5E00C5F0A2F733F8C3E8955E4002A85E88227E
:100B6E0088248825886122753A00753B7F2275C8D6
:100B7E0020A8CCA9CD75C824AA38AB3988388939B4
:100B8E00C3E89AF8E99BF9AA3AAB3BAC3AAD3B7E87
:100B9E00047F02C3EB940440021E1FC3EB94084073
:100BAE00021E1FC3ED13FDEC13FCDEF7C3EA9CFA25
:100BBE00EB9DFBEF6009C3E913F9E813F8DFF7EAE1
:100BCE0028FAEB39FB8A3A8B3B400122753AFF75C6
:100BDE003BFF2230600261E1854C50854D51D26061
:100BEE0043E680227892E6FFC3E535948240010FFA
:100BFE00C3E53594A040010FC3EF940640027F0574
:100C0E007E021E3072010EC3E53B940350060E0E9B
:100C1E003072010EC3E53B940250060E0E30720187
:100C2E000EA93BA83A7A04C3E913F9E813F8DAF7E8
:100C3E00C3E89EF8E99400F94009C3E89402E994E8
:100C4E000050047802E4F9E9FBE8FAC3E913FDE881
:100C5E0013FC884C894DC3EF94036037EF20E00DF1
:0F0C6E00E82CF8E93DF9ECFAEDFB020C8EE828D2
:100C7D00F8E939F9C3E89402F8E99400F97A02E445
:100C8D00FBC3EF9403400D8A4E8B4F884889498CE6
:100C9D004A8D4B22884E894F8A488B498C4A8D4B01
:100CAD002230600281AED26043E680E52D540660AD
:100CBD0027A83AA93BE53494085006E820E002A99C
:100CCD004D759100C3E498F594E499F595759104EB
:100CDD00D26053917F43E68022D265753D00752029
:100CED0000020CF9D265753D00752040E52D5406C6
:100CFD006002C265D2AF206005E53D60012278013A
:100D0D007A02C3E53B940540027802C3E53B940AA1
:100D1D0040027803C3E53B940F40027A0330690427
:100D2D00781E7A01206007E53D6003D2AF22D2AF75
:100D3D000000C2AFC3E53BFB940F40027B0FEB04F9
:100D4D003073012320620123F93069027982E58B2A
:100D5D00C39940D0053DEAFBE59BF45440B5200412
:100D6D00DBF6A19520650281F9C265759100AE3A59
:100D7D00AF3BC3E49EF594E49FF595759104D26065
:100D8D0053917F43E68081F930650281F9D895D280
:100D9D00AF2230690B0534206016753400020DBD8D
:100DAD0020600D20650A206B07158115810215FF46
:100DBD0022A84EA94F75910053917FC3E498F594E5
:100DCD00E499F595759104854850854951D2604354
:100DDD00E6802278003064053065027801E53575CE
:100DED00F007A4F9E5F028F5F0E9A2F013A2F1134C
:100DFD00A2F213F535C394785003753578C3E535F4
:100E0D0095364008D266C292C291C290306002C13E
:100E1D0019854A50854B51D26043E68022C2AFC23C
:100E2D0093C294C29530720B9001FF7406D5E0FD0C
:100E3D00020E68E53B54F86022E525600A207D022C
:100E4D00D292307D02D2907406D5E0FD207D02C293
:100E5D0092307D02C2907406D5E0FD207D02D293C2
:100E6D00307D02D295759F10753C02020FE7C2AF1F
:100E7D00207D02C290307D02C2923072179001DC4B
:100E8D00C294207D02C295307D02C2937406D5E0D6
:100E9D00FD020EA490013F306206E5256002D2915D
:100EAD00207D03759F20307D03759F00753C0302E7
:100EBD000FE7C2AFC293C294C29530720B9001B9C5
:100ECD007406D5E0FD020EFDE53B54F86022E525E4
:100EDD00600A207D02D290307D02D2927406D5E058
:100EED00FD207D02C290307D02C2927406D5E0FDD8
:100EFD00207D02D295307D02D293207D03759F0017
:100F0D00307D03759F20753C04020FE7C2AFC2917F
:100F1D00307217900196207D02C293307D02C295EA
:100F2D00C2947406D5E0FD020F3A90012D30620E89
:100F3D00E525600A207D02D292307D02D290759F08
:100F4D0010753C05020FE7C2AFC293C294C2953033
:100F5D00720B90016B7406D5E0FD020F82E53B54D8
:100F6D00F86012E5256002D2917406D5E0FDC291BC
:100F7D007406D5E0FDD294207D03759F20307D034E
:100F8D00759F00753C06020FE7C2AF207D02C2922D
:100F9D00307D02C29030721F90022A207D02C293D2
:100FAD00307D02C295207D02C295307D02C29374C0
:100FBD0006D5E0FD020FC790015130620EE52560A8
:100FCD000A207D02D290307D02D292207D03759F42
:100FDD0000307D03759F20753C01306B131210029C
:100FED007406D5E0FD7406D5E0FDD293D294D2956A
:100FFD00C266D2AF2290012BC292C291C290C2930F
:10100D00C294C295C2622278807609087609087664
:10101D00040876010876030876FF08760B0876013A
:10102D00087601087601788C76010876FF0876FF40
:10103D000876FF0876FF0876FF0876030876FF0826
:10104D0076FF0876FF0876250876D008762808768C
:10105D00500876040876FF08760208760008767A3E
:0D106D000876FF087601227887E6FFC27240
:10107A00BF0302D2727888E6C394036008C27DE691
:10108A0030E102D27DC27E7889E630E102D27EC3A7
:10109A00EF94026008758E01D2730210AC758E004F
:1010AA00C273227880E6149000809378A1F6788142
:1010BA00E6149000809378A2F61102227886E6144C
:1010CA0090008D9378A3F611022222789CE6753659
:1010DA00FF75370CB402067536A075370AB40306D5
:1010EA0075368275370522227896E6FA7897E6FBF6
:1010FA00307F047A007BFFC3EB9AFCC394825002D0
:10110A007C82756F00056FEC856FF0A4C3E5F094DF
:10111A008040F222D27F11F21206D57A007B007C3F
:10112A00101206CBE5592AFA74003BFBDCF37C0467
:10113A00C3EB13FBEA13FADCF7FEC27F11F222E5D6
:10114A00EF20E6037520000520903FFFE52014609C
:10115A0006901DFF1460009304600375EF12C2D35A
:10116A0053D9BF7581C043FF801206C675EF02438B
:10117A00B203E5B3240420E702F5B311027580FF38
:10118A0075A40075F1D475D4EF7590C075A53F7537
:10119A00F2FF75D50075A60175E241111412162EDB
:1011AA0078988670C2AF1206DF1206EF1206D512C1
:1011BA0006F61206D51206FD1206D5C2AFE4F8F6F7
:1011CA00D8FD78C879C8308407D9FBD8F7021C0043
:1011DA00111412162E117411AD11C611D411D51194
:1011EA00F111F27898867011027588507589127516
:1011FA00C82475910475D84075A82275B80275E699
:10120A0090759B80759D0075D10E75BC5875BB0392
:10121A0075BA1175E8801206C6D2AF1209E643DA2A
:10122A0001C2D8C2711206DF753001D2617B037A1E
:10123A000CE55870067A0CDB0221C51206D520701F
:10124A000221C5C270E559C3940240E3E52F541F39
:10125A00855B5AF55BB55AD7DAD7C26153DACF2024
:10126A007E0343DA20307E0343DA10C2D8C271C249
:10127A00757528001206DA307409C3E528940A4005
:10128A0002D2751206CB78023074027800C3E5598F
:10129A009840F0C2AF1206EF1206EF1206EFD2AF75
:1012AA001206DF7546007888E6B40302618C1206DE
:1012BA00CB788CE6C39401500302138CE530C394B7
:1012CA0001500302138C207435C3E55994FF50036F
:1012DA0002138CC2AF120704D2AF1206DAC3E55961
:1012EA00940150EFC2AF1206EF1206D01206EFD2E7
:1012FA00AF1206DAC3E55994FF40E90217D57F0217
:10130A00D27F11F21206DAC2AFC27F11F2AE59C30E
:10131A00E559947FD2AF40741206C6C2AF120704D1
:10132A00D2AFDFDC311EC3EE94057897F61206DFE2
:10133A0012166F1217587F0AD27F11F21206DAC2FA
:10134A00AFC27F11F2AE59C3E559947FD2AF50E6CE
:10135A001206C6C2AF1206EF1206D01206EFD2AFBD
:10136A00DFD6311EEE24057896F61206DF12166FC6
:10137A001217871206DA11F2C3E55994FF40F402F4
:10138A0017D5C3E559954640038559461206DA78BA
:10139A00017988E7B403027805C3E5599840024108
:1013AA00B0C2AF120704120704120704D2AF120622
:1013BA00DF753000E4F531F5320531E531F4703985
:1013CA000532789AE67819146012783214600D782A
:1013DA007D14600878FA146003753200C3E5329808
:1013EA00401715327531B478998670C2AF12070466
:1013FA00D2AF789886701206DA1206D0E5297005FF
:10140A0030740221C578012074027806C3E5599820
:10141A0040A77888E6C3940360031206DAE52970C8
:10142A000221C5C2AF1102E4F522F523F524F52500
:10143A00D2AF78858662F53EF53FF540F541F54233
:10144A00F56DF547F52CF52DF535120B75756D080B
:10145A0075BB101206C6120A81E5E820ECFBA8BD8E
:0E146A00A9BEE97001F8886E120A85756D083A
:1014780075BB107887E6FE760211747887EEF6C29F
:10148800AF755EFF120B5785225E85225F8522604D
:10149800D2AF752201752401752501855D647565D6
:1014A80001D268D269753400120F54120F96120BCC
:1014B80075120B7C120BF20214CC11021174756DAB
:1014C8000075BB03120CF1120D9F120DBE1207EE30
:1014D800120DE0120E2A120B7C120BE1120BF21203
:1014E8000CAE120CE6120D9F120DBE12084C12091A
:1014F800AA120DE0120E7B120B7C120BE1120BF2FA
:10150800120CAE120CF1120D9F120DBE12088512AC
:101518000DE0120EBF120B7C120BE1120BF2120C33
:10152800AE120CE6120D9F120DBE1208E2120DE06B
:10153800120F19120B7C120BE1120BF2120CAE12E5
:101548000CF1120D9F120DBE120947120DE0120F79
:1015580054120B7C120BE1120BF2120CAE120CE6B9
:10156800120A81120D9F120DBE120A85120DE01289
:101578000F96120B7C120BE1120BF2120CAE3069B3
:1015880038206B3585615E85615F855D64756501B1
:1015980079327A0AC3E534994012C269D26A8A3329
:1015A80085615E755FFF7560200215C1C3E55994BA
:1015B8000140030214CC0215FF306A1E206B1BE5A4
:1015C80033147007C26A755EFF81C2F533C3E559EB
:1015D800940140030214CC0215FFC3E55C94FA5051
:1015E80016307404E529600FC3E53B78F0306B02D0
:1015F800786098500281CCC2AF11027887E6FE76F7
:101608000211747887EEF6E4F522F523F524F52522
:10161800F562C268D2AF1206C61102307406E52917
:10162800700221C561BE901A0D78201216B1E5200E
:10163800B4550CA31216B1E520B4AA0302164F1133
:101648001412166F02166E901A0378807B0A12160F
:10165800B1A308DBF9901A0F788C7B151216B1A389
:1016680008DBF9901A2422C2AF1216F01216CA909B
:101678001A00740D1216B6A374021216B6A37413C8
:101688001216B6901A0378807B0A1216B5A308DBE7
:10169800F9901A0F788C7B151216B5A308DBF9128E
:1016A80017031216E1901A2422E493F622E6438FD8
:1016B80001538FFD75EF0275B7A575B7F1F0538F1C
:1016C800FE22438F02438F0175EF0275B7A575B7E8
:1016D800F1901A0DF0538FFC22901A0D7455D1B663
:1016E800901A0E74AAD1B6227A3079D07820901A3E
:1016F80040D1B1E520F709A3DAF7227A3079D09002
:101708001A40E7D1B609A3DAF922AB71A872BB0176
:10171800027980BB02027981BB03027982BB040291
:101728007984BB05027983BB06027986BB070279F7
:1017380092BB08027987BB0902799CBB0A027988A7
:10174800BB0B027989E8F7227C051206DFDCFB2255
:10175800C2AF1206EF1206F61206FD1207041206B1
:10176800D01206EF1206F61206FD1207041206D072
:101778001206EF1206F61206FD120704D2AF22C2B5
:10178800AF1207041206FD1206F61206EF1206D073
:101798001207041206FD1206F61206EF1206D01200
:1017A80007041206FD1206F61206EFD2AF22AE713A
:1017B800AF72C2AF1206EF1206EF1206EF1206D092
:1017C800DEF21207041206D0DFF8D2AF22F158F188
:1017D80050F150757101757201757300F1B67C0591
:1017E800AD591206DFC3ED955970F5C3E55994015B
:1017F800400AC3E55994FF40370218151217121210
:10180800166F121758C2AF75EF12121750DCD105B8
:1018180073C3E5739403500280C21217500572E532
:10182800711490009A93F808C3E57298500280A941
:101838001217501217500571C3E571940C500280AD
:0F1848009512101412166FC2AF75EF12121750CF
:101A00000D02130909040103FF0B01010155AA018D
:101A1000FFFFFFFFFF03FFFFFF25D0285004FF0259
:051A2000007AFF01FF48
:101A400023484B696E67313041232020202020201D
:101A500023424C48454C4923463333302320202031
:101A60002020202020202020202020202020202076
:101C0000C2AFC2D353D9BF7581C043B20343FF8073
:101C1000752438752503B1BF75EF0275E24043F1B5
:101C20001053A4EFD284780379E67C1075220075F6
:101C30002300901DCC7B0675249875250130840205
:101C4000813D208408D8FBD9F9DCF781AD308408C8
:101C5000D8FBD9F9DCF781ADB17FE493A3C39A60D7
:101C6000028126DBDDB171600281267B08E493FAF4
:101C7000A3B152DBF87A30B152752200752300B15E
:101C800071EAFCEBFDC3ED94FE400EB1718A278B27
:101C900028ED30E0048A828B83B1717AC270D8C398
:101CA000ED94FE601050CEBD0022EC600675200061
:101CB0000200008100A827A9280809D804D90281B8
:101CC000C9B175EA89AAF281BB0D8199C3ED94036C
:101CD0005049EDA2E092007AC5C3E5829400E58305
:101CE000941C5093200010438F02438F0175B7A5B9
:101CF00075B7F1F030001FA827A9280809438F0104
:101D0000538FFDD804D902A11689AAE275B7A5752B
:101D1000B7F1F0A3A103538FFC81757AC1BD030C09
:101D2000E493A3FAB136DCF8B12E81758177AA224B
:101D3000AB23B152EBFAEA6222752608C3E52313FE
:101D4000F523E52213F52250066323A0632201D573
:101D500026EAB1BFB1BF75260AEAF4200102D28497
:101D6000300102C284B1BFC3134002C201D526EBC9
:101D700022B175EAFB208402A175308402A17A7534
:101D80002608AE24AF25C3EF13FFEE13FEB1C3B197
:101D9000BFC3EA133084024480FA30E703632201B0
:101DA000C3E52313F523E52213F52250066323A090
:101DB000632201D526D9E52265236523F52222AECB
:101DC00024AF250E0FDEFEDFFCD20122424C486517
:0A1DD0006C6934373132F33006013C
:00000001FF
